:100000000C94AF010C94E7010C94E7010C94E70108
:100010000C94E7010C94E7010C94E7010C94E701C0
:100020000C94E7010C94E7010C94A71C0C94791D27
:100030000C949B170C94E7010C94E7010C94E701D6
:100040000C94E7010C94E7010C94E7010C94E70190
:100050000C94E7010C9423180C94E7010C94E7012D
:100060000C94E7010C94E7010C94E7010C94E70170
:100070000C94E7010C94E7010C94E7010C94E70160
:100080000C94E7010C94E7010C94E7010C94E70150
:100090000C94E7010C94E7010C94E7010C94E70140
:1000A0000C94E7010C94E7010C94E7010F040F0492
:1000B0003B043B04A304C104D905D905CC04650560
:1000C00076057605E61D0D1E051F0D1E051F591E22
:1000D0007C1E051FD31EE21E53005400550056001F
:1000E00035001E001F0020002100220023002400F4
:1000F0002500260027002D002E002A005F0060004A
:10010000610057002B0014001A00080015001700AA
:100110001C0018000C00120013002F0030003100EA
:100120005C005D005E003900040016000700090055
:100130000A000B000D000E000F00330034002800F1
:1001400059005A005B005800E1001D001B0006002A
:100150001900050011001000360037003800E500D6
:1001600062006300E000E300E2002C000151E700C0
:100170006500E40000000000000001000100010033
:10018000010001003A003B003C003D003E003F0002
:100190004000410042004300440045004C00010083
:1001A0000100010001000100010001000100005CEC
:1001B0000100010001000100010001000100010037
:1001C0000100010001000100010001000100010027
:1001D0000100010001000100010001000100010017
:1001E0000100010001000100010001000100010007
:1001F00001000100010001000100010001000100F7
:1002000001000100010001000100010001000100E6
:100210000100010001000000000000002203730043
:100220006F007500740068007000610077002000A6
:10023000640065006600610075006C0074000000D9
:100240001003640072006500770067007500790094
:1002500000000403090409023B00020100A0FA099E
:1002600004000001030101000921110100012240E5
:1002700000070581030800010904010001030000D3
:1002800000092111010001227B00070582032000E3
:100290000112010002000000084F48505301000104
:1002A00002000105010902A10185020901A1000561
:1002B0000919012908150025019508750181020514
:1002C00001093009311581257F95027508810609DC
:1002D000381581257F950175088106050C0A3802BD
:1002E0001581257F950175088106C0C0050109802B
:1002F000A101850319012AB700150126B700950150
:1003000075108100C0050C0901A101850419012A9D
:10031000A002150126A002950175108100C00501FB
:100320000906A101050719E029E71500250195082F
:10033000750181029501750881010507190029FFE2
:10034000150026FF0095067508810005081901298A
:1003500005950575019102950175039101C0112460
:100360001FBECFEFDAE0DEBFCDBF04B603FE18C07C
:100370008091980290919902A0919A02B0919B026B
:100380008730904BA740B04B59F4109298021092CE
:10039000990210929A0210929B02E0E0F8E309950C
:1003A00011E0A0E0B1E0E0E7FFE302C005900D92AC
:1003B000AE38B107D9F722E0AEE8B1E001C01D9236
:1003C000A839B207E1F70E94E4110C94B61F0C940F
:1003D000000081E0089581E008950C94EB010895F8
:1003E0000C94EF011F93CF93DF9300D000D01F92A6
:1003F000CDB7DEB749835A836B83309191018981F0
:100400009A81311114C0662359F0222349F00E94C9
:100410001608182F682F89819A810E94BF0703C090
:100420000E94EA07182F69817A81812F04C00E94F7
:10043000160869817A810F900F900F900F900F909E
:10044000DF91CF911F910C944C0FFC01262F40811E
:1004500051816281738184810C94F20181E008955D
:10046000CF93DF93EC0160E00E942502BE01DF9193
:10047000CF910C94F0010C9495100C949110089568
:100480000E9469060E943F022FEF84E39CE0215006
:1004900080409040E1F700C000000C9449180F9391
:1004A0001F93CF93DF938C0161E00E942502EC0142
:1004B000B8010E94ED018823F1F1B801CE010E943C
:1004C00066168823C1F1B801CE010E947A148823F0
:1004D00091F1B801CE010E94C215882361F1F801A3
:1004E0008281882309F1CB358DE5D807C1F050F41E
:1004F000C115FCE5DF0781F0CF3DDC45A9F40E9482
:100500004D0D19C0CC35EDE5DE0761F0CD35DD458B
:1005100059F40E94900C08C00E9440020CC00E9436
:10052000990C02C00E949C0CC801DF91CF911F91D1
:100530000F910C94E90180E0DF91CF911F910F9111
:1005400008950E947D170C94BA020E94BD020C947B
:10055000831708950C94A90281E008950C94AC02CD
:100560000895CF93C82F0E94AA028C2F0E94AE023A
:10057000CF91089580E00C94B1020E94C2160C94B1
:10058000B1020E94C21690919001891721F08093C8
:1005900090010C94B1020895CF93DF93CDB7DEB7ED
:1005A0002B970FB6F894DEBF0FBECDBF4F83588791
:1005B00069877A878B8761110E94DC0B9E012F5F10
:1005C0003F4F86E0F90111928A95E9F785E0FE0137
:1005D0003796D90101900D928A95E1F789819A8128
:1005E0004C815D81452B31F09F3F31F491E08F3F8D
:1005F00019F403C091E001C090E090FF09C0498167
:100600005A816B817C818D819E810E94FD0A05C08B
:10061000C9010E942E028111F2CF2B960FB6F894D9
:10062000DEBF0FBECDBFDF91CF910895FC01808169
:1006300091810E9458080895CF93882309F450C0EF
:10064000C82F8CEF8C0F813AD0F46C2F809102016F
:10065000909103010E941F17882349F06C2F80910D
:100660000201909103010E9457170E94FE0B6C2F0C
:1006700080910201909103010E9455170CC080E205
:100680008C0F883058F4C77081E001C0880FCA957C
:10069000EAF70E94BF0BCF910C94FE0BEBE5EC0F39
:1006A000E33040F4F0E0E95BFE4F808190E0CF91D1
:1006B0000C94E716E8E5EC0FE73150F4F0E0EE0FAC
:1006C000FF1FE75EFE4F80819181CF910C94FD1654
:1006D000CD3E30F08C2F0E946912CF910C943B13C9
:1006E000CF910895882389F19CEF980F913A40F4B7
:1006F000682F80910201909103010E9457170DC04D
:1007000090E2980F983058F4877091E001C0990FEB
:100710008A95EAF7892F0E94C50B0C94FE0B9BE586
:10072000980F933020F480E090E00C94E71698E561
:10073000980F973120F480E090E00C94FD168D3EE8
:1007400020F00E94C4120C943B1308951F93CF9382
:10075000DF93182FEB010E941C03209741F08FE9D3
:100760009FE00197F1F700C000002197F6CF812F9D
:10077000DF91CF911F910C947203893319F060E0DF
:1007800070E002C060E570E00C94A603882321F0BD
:100790000E94BF0B0C94FE0B0895882321F00E9449
:1007A000C50B0C94FE0B0895CF92DF92EF92FF924F
:1007B0000F931F93CF93DF937C01D62FC72FFC019C
:1007C0001281058102950F700E94B50B8823B9F044
:1007D0001123A9F08C2F807F803421F080E28D0FCF
:1007E000883068F08091620282FD09C082E00E9438
:1007F0005E0C0E94B50B91E0D82ED92601C0D12CF9
:10080000CC2EC2948FE0C8228C2D90E08C309105C4
:1008100008F0CFC1FC01EA5AFF4F0C944D1F8C2FFA
:10082000807FCF70882311F0C295C07F112399F08B
:10083000CC2309F4AAC180E28D0F883010F0D111C9
:1008400004C08C2F0E94BF0B03C08C2F0E94CF0BC3
:100850000E94FE0B9AC18D2F0E947203CC2309F4D3
:10086000A8C180E28D0F883038F1DD2329F18C2F6B
:100870000E94D50B24C08C2F807FCF70803211F066
:10088000C295C07FDD2319F0D130A1F13DC0809128
:10089000620282FF17C0112349F0CC2329F08C2F6C
:1008A0000E94BF0B0E94FE0B80E070C180E00E949E
:1008B0007203CC2309F47DC18C2F0E94C50B0E94CA
:1008C000FE0B77C1112371F0002341F0013031F4A8
:1008D0000E94DF0B8C2B0E94E70B6BC10E94DF0B89
:1008E0008C2B1DC0002319F0013009F462C10E9455
:1008F000F40B25C0112321F0063008F05AC10EC0B8
:10090000053008F056C11BC0112361F0002331F0FF
:10091000F701858180FF39C18F7085838C2F0E94FC
:10092000C60347C1002359F0D93309F03FC1FFEF97
:1009300007EE13E0F15000401040E1F735C18C2F75
:100940000E94CD0336C18C2F86958695837019F051
:10095000813061F02EC1112321F08D2F9C2F9370D7
:1009600002C080E090E00E94E7162BC1112321F025
:100970008D2F9C2F937002C080E090E00E94FD16A6
:1009800020C18D2F112319F00E94691202C00E940C
:10099000C4120E943B1315C18C2F837009F047C00D
:1009A00011110BC12D2F229526952770220F220F92
:1009B0006D2F6F70862F90E0A0E0B0E0022E04C093
:1009C000880F991FAA1FBB1F0A94D2F7D4FF10C02B
:1009D0004FE050E060E070E004C0440F551F661F18
:1009E000771F2A95D2F7409550956095709503C072
:1009F00040E050E0BA01C695C695C3708A019B01DC
:100A0000082B192B2A2B3B2BC901B801C23049F006
:100A100058F4C13019F00E94D506CFC00E94C30619
:100A2000CCC00E94E706C9C00E94C106C6C01123FF
:100A300019F08C2F817001C08695882309F4BDC000
:100A40002D2F229526952770220F220F6D2F6F7064
:100A5000862F90E0A0E0B0E0022E04C0880F991F1E
:100A6000AA1FBB1F0A94D2F7D4FF10C04FE050E07A
:100A700060E070E004C0440F551F661F771F2A9581
:100A8000D2F7409550956095709503C040E050E0D6
:100A9000BA01C695C695C3708A019B01082B192B14
:100AA0002A2B3B2BC901B801C23049F058F4C130A0
:100AB00019F00E949A0781C00E9488077EC00E9498
:100AC000AC077BC00E94FB0678C0CF70112339F0C1
:100AD0008C2F0E9421078D2F0E94C6036EC08D2F80
:100AE0000E94CD038C2F0E94420767C0D23F21F1A4
:100AF00028F4D03F41F0D13FC1F043C0D33F19F1BA
:100B0000D43F79F03EC0112341F0053008F051C0C8
:100B10008C2F8F710E9467074CC0063008F049C0C7
:100B2000F7CF8091620282FF18C0112339F08C2F19
:100B30008F710E9421073DC01123C9F38C2F8F7143
:100B40000E94420736C0112329F08C2F8F710E941A
:100B50000C072FC00E9407072CC0112349F0CF714A
:100B60008C2F0E94210763E08C2F0E94430C21C030
:100B700081E00E945E0C0230E0F082E00E945E0C98
:100B800018C0112331F0002391F28D2F0E941C0315
:100B900010C0002399F2D93349F41FEF27EE33E058
:100BA000115020403040E1F700C000008D2F0E941E
:100BB000720388EF8C0D843020F40E94C2160E94CC
:100BC000B102DD20C9F00E94B10B80FD15C0F70114
:100BD00012820E94AB0B0E942107C7010E941D06D2
:100BE0000E94AB0BDF91CF911F910F91FF90EF907F
:100BF000DF90CF900C944207DF91CF911F910F911E
:100C0000FF90EF90DF90CF9008950F931F93CF93B5
:100C1000DF93EC01688179818A810E9463088C01ED
:100C20000E94BE070E94AF06B801CE010E94D40305
:100C3000DF91CF911F910F910895CF93DF93EC0136
:100C4000988189812B813C81232B31F08F3F31F4B6
:100C500081E09F3F19F403C081E001C080E080FD86
:100C60001DC0CE010E944F02811110C00E94B50B21
:100C70008823A1F08A81882389F08091620282FD15
:100C80000DC082E0DF91CF910C945E0CCE010E94EA
:100C90000506CE01DF91CF910C943002DF91CF9108
:100CA000089580E090E00E94E71680E090E00E94C6
:100CB000FD160E94DC0B0E94FE0B0E946C140C942B
:100CC0003B1380910201909103010E9459170C94EB
:100CD00051060E94CC0B0C94610692959F70963041
:100CE00079F010F4925001C09A50923068F4803F2D
:100CF00069F018F4883E40F409C0843F29F406C026
:100D0000883E20F0813F11F080E0089581E0089551
:100D1000FC01808191810E9458080E946D0608950F
:100D2000CF93DF9300D000D01F92CDB7DEB70F90E6
:100D30000F900F900F900F90DF91CF910895CF9368
:100D4000DF9300D000D000D0CDB7DEB726960FB627
:100D5000F894DEBF0FBECDBFDF91CF910895089507
:100D600008950C94B0060C94B1060E94B3066093EB
:100D7000CD017093CE018093CF019093D0010C945C
:100D800051060C94B5060F931F930091CD0110915D
:100D9000CE012091CF013091D001602B712B822B9D
:100DA000932B1F910F910C94B5060F931F930091F5
:100DB000CD011091CE012091CF013091D00160235F
:100DC0007123822393231F910F910C94B5060F93E7
:100DD0001F930091CD011091CE012091CF01309150
:100DE000D00160277127822793271F910F910C94C0
:100DF000B5060C94B0060E94F9066093C901709381
:100E0000CA018093CB019093CC010C94510660E011
:100E100070E0CB010C94FB060F931F9341E050E070
:100E200060E070E08A019B0104C0000F111F221FC7
:100E3000331F8A95D2F7C901B8011F910F910C9405
:100E4000FB060F931F9341E050E060E070E004C0A8
:100E5000440F551F661F771F8A95D2F78091C901ED
:100E60009091CA01A091CB01B091CC018A019B0164
:100E7000082B192B2A2B3B2BC901B8011F910F916D
:100E80000C94FB060F931F9341E050E060E070E08C
:100E900004C0440F551F661F771F8A95D2F74095EF
:100EA0005095609570958091C9019091CA01A0916B
:100EB000CB01B091CC018A019B01082319232A237D
:100EC0003B23C901B8011F910F910C94FB060F93AE
:100ED0001F9341E050E060E070E004C0440F551FF4
:100EE000661F771F8A95D2F78091C9019091CA0138
:100EF000A091CB01B091CC018A019B010827192751
:100F00002A273B27C901B8011F910F910C94FB06BA
:100F10000F931F930091C9011091CA012091CB0139
:100F20003091CC01602B712B822B932B1F910F9151
:100F30000C94FB060F931F930091C9011091CA01F5
:100F40002091CB013091CC01602371238223932324
:100F50001F910F910C94FB060F931F930091C901F1
:100F60001091CA012091CB013091CC0160277127EB
:100F7000822793271F910F910C94FB06089529E077
:100F8000929F800D1124E82FE695E695E6958770EF
:100F900051E001C0550F8A95EAF785E0E89FF0011E
:100FA0001124EE56FE4F20E030E070E04081CB018E
:100FB000022E02C0969587950A94E2F7817081957A
:100FC00084278523842781932F5F3F4F2530310568
:100FD00069F7089529E0929F800D1124682F669586
:100FE00066956695982F977085E0689FB0011124EB
:100FF00040E050E080E0FB01E40FF51FEE56FE4FAD
:10100000208130E0092E02C0369527950A94E2F738
:1010100021703327042E01C0220F0A94EAF7822B95
:101020004F5F5F4F4530510531F70895BF92CF9222
:10103000DF92EF92FF920F931F93CF93DF938C0178
:10104000C090C901D090CA01E090CB01F090CC01D2
:101050008091CD019091CE01A091CF01B091D001AE
:10106000C82AD92AEA2AFB2ACFE1D0E0D701C60153
:101070000C2E04C0B695A795979587950A94D2F73C
:1010800080FD04C0219790F7B12C07C0BC2EB80199
:101090008C2F0E945F0F0197A9F38B2DDF91CF91C9
:1010A0001F910F91FF90EF90DF90CF90BF90089528
:1010B000CF93DF93EC010E941608BE010E945F0FE0
:1010C000DF91CF9108951F93CF93DF93EB01909120
:1010D0009101992321F0CB010E94580813C0882365
:1010E00049F0CB010E941608182F682FCE010E94EC
:1010F000BF0704C0CB010E94EA07182FBE01812F51
:101100000E945F0FDF91CF911F9108951F93CF939E
:10111000DF93C091D10116E08091D201C81799F0F8
:10112000D0E01C9FF0011D9FF00D1124ED52FE4FE9
:101130004081518162817381848195810E949F06E3
:101140002196C770E9CFDF91CF911F91089540910B
:101150000302509104026091050270910602809191
:101160000702909108020C949F06EF92FF920F9352
:101170001F93CF93DF938091080282958F7009F0BF
:1011800065C080910502882309F460C08091D10177
:10119000F090D201109103020091040260910602C6
:1011A0007091070291E01F3F09F090E0C0910001AB
:1011B000D0910101292F96E0E92E8F1509F446C040
:1011C0006115710521F00F3F21F030E003C031E0DF
:1011D00001C0322F90E030FD36C0E89EF001E99E5C
:1011E000F00D1124DF01AD52BE4F11963C911197C5
:1011F000301329C03C91311326C012963C911297AE
:10120000311121C013964D915C911497461B570BD9
:101210004C175D07C0F4809108028F708061809345
:101220000802E852FE4F80818F708061808383E0E6
:1012300092E00E941D06DF91CF911F910F91FF90C8
:10124000EF900C94860801968770B7CFDF91CF910D
:101250001F910F91FF90EF9008959F92AF92BF92D0
:10126000CF92DF92EF92FF920F931F93CF93DF9372
:10127000CDB7DEB761970FB6F894DEBF0FBECDBF16
:101280008C0185E0F801DE011D9601900D928A9592
:10129000E1F7D8011296EC9090910302E0910402DC
:1012A00020910602309107022115310531F0EF3F00
:1012B00031F481E09F3F19F403C081E001C080E078
:1012C000B82FB1709B2E80FD47C1D8014C9111966B
:1012D0005C9111971396AD90BC90149783E0C82E43
:1012E00082E0D82EF0900502B501621B730B2091AD
:1012F000000130910101FF2009F4D9C0809108025A
:101300006217730708F095C0282F207F09F052C09C
:101310005E1313C0491311C0FE2CE1100EC08F7074
:101320008061809308020E94A708C6010E941D06E2
:1013300080910802F80185834DC1AB2831F05F3FF1
:1013400031F481E04F3F19F403C081E001C080E037
:1013500080FD03C081E08E2502C080E090E0F82F80
:10136000F170FF2E80FF1CC08091D1012091D2012D
:1013700036E0821709F40BC190E0389FF001399FE5
:10138000F00D1124ED52FE4F6181561306C06081AD
:10139000461303C06281E61203C001968770E9CF4D
:1013A000FE2CEE2009F416C1809108028160809322
:1013B000080254C05E1306C0491304C0E11002C005
:1013C000F80199C0C8010E948806882361F1EE20C7
:1013D00051F120910802822F82958F7090E0029740
:1013E00074F0809103029091040298878F8319868C
:1013F000BB86AA862C87CE0107960E941D0686E032
:10140000F801A3E0B2E001900D928A95E1F70E9405
:10141000B5080E94A7080AC05E1711F1C8010E9412
:10142000880681112CC0C8010E941D06FF24F39478
:10143000D1C0282F207F81F77A2DB98AA88A6E2DF6
:1014400089890E94900683E092E00E941D0686E052
:10145000D6011D928A95E9F70E94A708F12CBAC01F
:101460004913DCCFE110DACFF8018583C8010E946F
:101470001D0686E0D6011D928A95E9F7ABC0EE20E5
:1014800091F220910802822F82958F7090E002974E
:101490000CF4B5CF80910302909104029A83898362
:1014A0001B82BD82AC822E83CE010196A6CF62172D
:1014B000730708F044C0FE2CEE2009F4B4CF5E138D
:1014C00030C049132EC02091080220FD21C0822F78
:1014D00082958F70482F50E041155105C9F0F801F1
:1014E00025834F30510541F08F5F982F9295907F63
:1014F000822F8F70892B8583C8010E941D0686E08C
:10150000F801A3E0B2E001900D928A95E1F73CC0AA
:1015100086E0F801A3E0B2E001900D928A95E1F730
:1015200059C0C8010E948806811169CF80910802C4
:10153000816080930802C8010E941D064BC07A2D6D
:10154000B98AA88A6E2D89890E94900686E0D60104
:101550001D928A95E9F718C0EE2009F464CFC801FE
:101560000E948806F82E882309F45DCF86E0F801F2
:10157000A3E0B2E001900D928A95E1F783E092E05A
:101580000E9416030E94B5080E94A70823C04D8739
:101590005E878D859E850E945808292F22952F7081
:1015A000223028F49F7039F0811105C00BC024301F
:1015B00028F49F7049F4805E883020F0C8010E94B2
:1015C0001D069F2CF92C06C0D80115969C91907F82
:1015D00091F7F8CF8F2D61960FB6F894DEBF0FBE4E
:1015E000CDBFDF91CF911F910F91FF90EF90DF90D2
:1015F000CF90BF90AF909F9008951F93CF93DF93AC
:10160000CDB7DEB72C970FB6F894DEBF0FBECDBFB7
:101610004F83588769877A878B879C87CE01079687
:101620000E942D098823D1F09F8188852A853B85DA
:10163000232B31F08F3F31F481E09F3F19F403C039
:1016400081E001C080E080FD47C04F8158856985F9
:101650007A858B859C850E949F063EC086E0FE01B0
:101660003796DE01119601900D928A95E1F7FF8180
:10167000E8856A857B856115710531F0EF3F31F4AE
:1016800081E0FF3F19F403C081E001C080E080FDEC
:1016900023C02091D20130E0C901019687709927BB
:1016A0004091D10150E084179507F1F1F983EA8365
:1016B0007D836C8396E0929FD001939FB00D11249F
:1016C000AD52BE4FFE01319601900D929A95E1F711
:1016D0008093D2010E94860816E08091D1019091FA
:1016E000D201891771F1189FC00111248D529E4FAC
:1016F0000E942D09882329F1E091D1011E9FF0015C
:101700001124ED52FE4F40815181628173818481A9
:1017100095810E949F068091D10190E0019687708B
:1017200099278093D101D9CF0E9469061092D201E6
:101730001092D101E3E0F2E086E0DF011D928A958C
:10174000E9F72C960FB6F894DEBF0FBECDBFDF9140
:10175000CF911F910895809111028595859585956A
:1017600008958091110287700895909111029770E9
:1017700081E009F480E0089580911C020895909121
:101780001C02892B80931C020895809590911C0265
:10179000892380931C02089510921C020895909151
:1017A0001B02892B80931B020895809590911B0248
:1017B000892380931B02089510921B020895809143
:1017C0001202089508950C94E20B0C94E30B90918F
:1017D000620292FD08C090911202981721F0809346
:1017E00012020C94E50B089580911202882329F0CF
:1017F0001092120280E00C94E50B0895CF93DF93D2
:10180000E0910201F091030180911C028083E0913C
:101810000201F0910301908180911B02892B80834A
:1018200080911202882381F0E0910201F09103017E
:101830009081892B808380910201909103010E9405
:10184000131781110E94F40BC0910201D091030182
:1018500048E050E069E072E0CE010E94671F892BEA
:1018600069F088E0FE01A9E0B2E001900D928A954E
:10187000E1F7CE01DF91CF910C94CE16DF91CF919D
:1018800008950C94E20B9091620292FD10C098E0D2
:10189000899F90011124262B209311020E94210779
:1018A000809111028595859585950C94410C0C9439
:1018B00021071092110280E00C94410C209111023A
:1018C0008095822380931102982F977099F430E0CD
:1018D000482F082E000C550B2417350759F090910E
:1018E000620292FD07C08595859585950E94420705
:1018F0000C94590C08959091620292FB222720F9D2
:10190000281769F080FB92F990936202809161023E
:10191000909162020E94C90C82E00C945E0C0895C2
:101920008091620282FB882780F991E089270C94DC
:101930007B0C81E00C947B0C80E00C947B0C6FEFB3
:101940007FEF80E090E00C94A01F80E090E00E9488
:101950007C1F21E0893E9E4F09F020E0822F0895F0
:1019600082E090E00C94741F83E090E00C94741F6C
:10197000CF9384E090E00E94741FC82F82E290E031
:101980000E94741F2C2F30E0A901582BCA01CF915F
:101990000895CF93C92F682F84E090E00E94821FA2
:1019A0006C2F82E290E0CF910C94821FAB01BC01BE
:1019B0008FE090E00C94941FAB01BC0183E190E0B8
:1019C0000C94941F60E070E0CB010C94DC0C60E0A0
:1019D00070E0CB010E94D60C0C94E20C69EE7EEF15
:1019E00080E090E00E94A01F60E082E090E00E9412
:1019F000821F60E083E090E00E94821F1092CD0180
:101A00001092CE011092CF011092D00160E084E0DC
:101A100090E00E94821F60E082E290E00E94821FBC
:101A200060E085E090E00E94821F60E086E090E048
:101A30000E94821F6FEF87E090E00E94821F40E0CB
:101A400050E0BA0188E090E00E94941F60E08DE0D1
:101A500090E00E94821F40E050E0BA0188E190E0EF
:101A60000E94941F60E087E190E00E94821F40E0A6
:101A700050E0BA018CE190E00E94941F60E070E0B9
:101A800080E290E00E94A01F40E050E0BA0188E1AF
:101A900090E00E94941F0C94E70C0C94EE0C682FBD
:101AA0008EE090E00C94821F0E940818609333022D
:101AB00070933402809335029093360260932F0224
:101AC000709330028093310290933202089585B76B
:101AD000806885BF85B7806885BF089581E00895D7
:101AE0000C946E0D08950C94720D0C94720D0C9460
:101AF000750D0C94720D0C94790D0C94720D0E945E
:101B0000670D8BE390E10E94B8160E947D0D0C9446
:101B10007B0D0E94730D0C94720D0E9458100C9452
:101B2000B0020E94F3170E943D110E948D0D0C948B
:101B3000770D5F926F927F928F929F92AF92BF923A
:101B4000CF92DF92EF92FF920F931F93CF93DF9389
:101B5000CDB7DEB72A970FB6F894DEBF0FBECDBF64
:101B60000E945211C82E81110E94540D3DE1832E16
:101B700032E0932E00E010E0502E802F0E947C1067
:101B80005C01F401619071904F016826792661141F
:101B90007104B1F40F5F1F4F0930110569F78FEF22
:101BA00089838A831B820E94FC178160782F9D8322
:101BB0008C8349815A816B818D810E94CC023AC00D
:101BC0008091370281FD0E948510D12CEE24E39490
:101BD000F12CC3018E219F21892B29F10E94700DC8
:101BE0008823A9F0DE825F82AE20BF2081E0AB288F
:101BF00009F480E088870E94FC178160782F9A871B
:101C000089874E815F8168858A850E94CC02000F9A
:101C1000111FF801E35EFD4F80819181E826F926CE
:101C2000F182E08207C0D394EE0CFF1CF9E0DF12D2
:101C3000D0CFB0CF81E0C11001C080E02A960FB6AE
:101C4000F894DEBF0FBECDBFDF91CF911F910F91F2
:101C5000FF90EF90DF90CF90BF90AF909F908F90CC
:101C60007F906F905F9008950E94990D0E94591384
:101C70000C94C102CF93DF930E94640FEC01811595
:101C800021E5920708F045C0811530E5930708F07B
:101C900094C0883E910528F5803E910508F0F8C073
:101CA000883A910570F4853A910508F07CC081303E
:101CB000910509F475C008F4E8C0049708F0E8C07D
:101CC000E4C08F3B910508F0E0C0C85AD0E0CC0FCB
:101CD000DD1FC65BDE4F0990D881C02DCE01946414
:101CE000D8C0811540E2940758F4811551E095075A
:101CF00008F0CEC08D3E910508F4C7C09065C9C0FC
:101D0000C11580E4D80708F4C0C0DF70CE01906A26
:101D1000C0C0811525E59207A8F4811534E5930725
:101D200008F095C0811543E5940708F07BC0811544
:101D300052E5950708F061C0D82FCC27CE01816FFE
:101D4000906AA7C0C11589E5D807A0F4C11528E598
:101D5000D20708F082C0C11536E5D30708F095C058
:101D60008C2F0E94F80F8F7190E0D82FCC27CE01D6
:101D700090628FC0C1154AE5D40708F474C0CE0143
:101D800090568115904208F080C08D2F8F710E946F
:101D9000F80FDD27D0628F71AE01582BCA0179C0D0
:101DA00081E090E076C0C55AD0E0C858DE4F888107
:101DB000C82FD0E0CE0190646CC074E096958795F2
:101DC0007A95E1F7282F23703C2F337081E090E063
:101DD00002C0880F991F3A95E2F79C68AC01522B1C
:101DE0009A019C2F9F709695969550E2959FE001E1
:101DF0001124C9018C2B9D2B4CC08370992721E0A5
:101E000030E002C0220F331F8A95E2F79C2F96958F
:101E1000969580E2989FE0011124C22BD32BCE012E
:101E20009C6837C08370992721E030E002C0220F00
:101E3000331F8A95E2F79C2F9695969540E2949FE2
:101E4000E0011124C22BD32BCE019A6822C0D82FD7
:101E5000CC27CE01846F906A1CC0DC2FCC27CE012A
:101E6000806F906A16C08C2F8F700E94F80F94E0DC
:101E7000D695C7959A95E1F7CF70D0E0DC2FCC27A7
:101E8000D0699E01282BC90104C080E090E001C008
:101E9000CE01DF91CF91089521E5829FC0011124E9
:101EA000FC0129E0729FE00DF11D1124E60FF11DE8
:101EB000EE0FFF1FE852FF4F8591949108950E9405
:101EC0004C0F0E943A0E08958238910569F1B0F4E2
:101ED0008133910509F46DC048F48932910509F404
:101EE00063C08A32910509F469C00895853391056C
:101EF00009F455C089339105B9F00895833E9105E1
:101F000069F138F4803E9105B1F0823E910509F106
:101F10000895863E9105A9F1873E9105B9F1843E69
:101F2000910509F064C023C02091610220FD4FC0DB
:101F300021FD4DC008958091610280FD44C08091D3
:101F4000620280FF44C08091610284FD42C083EE42
:101F50004DC08091610282FF38C0F5CF809161024F
:101F600082FD33C08091620280FD31C0ECCF809150
:101F7000620281FF32C08091610284FD2AC087EE37
:101F800035C08091610283FF26C0F5CF8091610248
:101F900083FD21C08091620281FD1FC0ECCF809142
:101FA000610285FD1CC01DC08091610285FD19C0C4
:101FB00016C08091610286FD16C017C08091610233
:101FC00086FD13C010C089E311C082EE0FC080EE01
:101FD0000DC080E00BC086EE09C084EE07C089E228
:101FE00005C085E303C08AE201C081E390E0089563
:101FF0009091610292FF0DC0282F2871283019F4AA
:10200000877F846006C0282F2471243011F48B7FD1
:10201000886093FF0DC0282F2871283119F4877E1E
:10202000846106C0282F2471243111F48B7E8861CD
:102030002091620220FF0DC0382F3871383019F41A
:10204000877F816006C0382F3171313011F48E7F67
:10205000886021FF0DC0282F2871283119F4877E50
:10206000816106C0282F2171213111F48E7E886193
:1020700094FD877E089580E008950C949F0C0E9443
:1020800052112FEF86E791E0215080409040E1F718
:1020900000C000000E94521180E00E947C1080FF6E
:1020A00004C00E943D100C94491808950C943F10F0
:1020B0000E94A50C811102C00E944D0D0E94B00C1F
:1020C000809337020E94B80C909362028093610261
:1020D0000E9456100E94B40C682F70E080E090E0DF
:1020E0000E94C1066091C9017091CA018091CB0123
:1020F0009091CC010C94F906E82FF0E0EE0FFF1F51
:10210000EB58FD4F808191810895089580EA8A956A
:10211000F1F7089500C008950C94861008950C946A
:102120008E100C948F100C948E100C949310F894C5
:10213000E82FE295EF70F0E031A1282F2F7081E0B9
:1021400090E001C0880F2A95EAF7982F9095932385
:1021500091A392A1892B82A3789408950F931F9342
:10216000CF93DF93C4E8D1E089918F3F11F00E94B3
:10217000971081E0CD38D807B9F7CBE7D1E004E874
:1021800011E089918F3F11F00E9497100C171D07E5
:10219000C1F7DF91CF911F910F910895BF92CF9218
:1021A000DF92EF92FF920F931F93CF93DF938C01F7
:1021B000C62FD0E0CE018C579E4F6C01FC01908160
:1021C0009F3F09F450C0B62EF894E92FE295EF70C6
:1021D000F0E081A19F7021E030E001C0220F9A95CC
:1021E000EAF7822B81A382A12095282322A3789449
:1021F0000E948A10EBE7F1E044E851E021E030E092
:10220000E12CF12C61916F3F89F0A62FA295AF7060
:10221000B0E090968C9190E06F7002C09595879594
:102220006A95E2F780FD02C0C90102C080E090E03B
:10223000E82AF92A220F331F4E175F0719F7F60114
:1022400080818F3F11F00E94971061E0E114F1044A
:1022500009F460E08B2D0E948C10CC0FDD1FC00FA5
:10226000D11FF982E882DF91CF911F910F91FF90EA
:10227000EF90DF90CF90BF9008950E94AE1082E162
:10228000E5E7F2E0DF01982F1D929A95E9F7E3E682
:10229000F2E0DF011D928A95E9F789E00E949D1125
:1022A0000C943B02FF920F931F93CF93DF93CDB714
:1022B000DEB762970FB6F894DEBF0FBECDBF8E01BA
:1022C0000F5F1F4F82E1F80111928A95E9F7F12C17
:1022D0006F2DC8010E94CE10F394F9E0FF12F8CFE1
:1022E00042E150E0B80183E692E00E94671FFF24BC
:1022F000F394009709F4F12C892B41F082E1F80165
:10230000A3E6B2E001900D928A95E1F72F2D49E006
:1023100065E772E083E692E00E949E110E943D0212
:102320008F2D62960FB6F894DEBF0FBECDBFDF9142
:10233000CF911F910F91FF9008950895FF920F93F1
:102340001F93CF93DF93F82E092F162FD72FC42F6B
:10235000222349F081E080933A020E94FC17909377
:1023600039028093380280913A028823D9F0809113
:102370003802909139020E941418059798F0EF2DB9
:10238000F02FA12FBD2F80E090E04C2F50E084175C
:10239000950734F4219131912D933D930196F7CF18
:1023A00010923A02DF91CF911F910F91FF90089503
:1023B0000E94FF190E94910D0C940B1A0E940F1A93
:1023C0000E94340E0C94291A0E949A170E94E61952
:1023D0000E947F0D0E94D8110E94DE110E94890D7B
:1023E000FBCF8091410280FF06C06091090170E03F
:1023F000660F771F26C081FF04C06091090184E049
:1024000005C082FF07C06091090188E0689FB001A4
:10241000112417C0909140029923D1F060910801D6
:10242000961788F72091090188E0289F90011124D0
:10243000929FA001939F500D112470E0CA010E9449
:10244000391F6038710540F46115710519F406C033
:1024500068E070E0862F08958FE7089581E0089581
:102460008091410280FF08C06091050170E0759580
:1024700067957595679521C081FF06C0609105013C
:1024800070E07595679519C082FF04C060910501E1
:1024900070E010C090913F02992399F0609104017F
:1024A0009617A0F780910501899FC001112470E063
:1024B0000E94391F6038710540F46115710519F4E7
:1024C00006C061E070E0862F08958FE7089581E0EF
:1024D00008958D3E21F40E94F111819504C08E3E35
:1024E00029F40E94F1118093450208958F3E21F452
:1024F0000E94F111819504C0803F29F40E94F111DE
:10250000809344020895893F19F40E94301205C057
:102510008A3F31F40E9430128195809346020895DB
:102520008B3F21F40E943012819504C08C3F29F426
:102530000E9430128093470208959FE0980F9830D0
:1025400078F421E030E0A90102C0440F551F9A95AC
:10255000E2F7CA0190914302892B809343020895C8
:102560008D3F21F48091410281600BC08E3F21F4A8
:1025700080914102826005C08F3F29F48091410221
:1025800084608093410208958D3E39F49091450214
:1025900097FF35C01092450259C08E3E29F49091A4
:1025A00045021916BCF32BC0909144028F3E29F4CA
:1025B00097FF25C01092440249C0803F19F41916B4
:1025C000CCF31DC090914602893F29F41916BCF442
:1025D000109246023BC08A3F19F497FF10C0F8CF13
:1025E0008B3F39F49091470297FF09C01092470240
:1025F0002DC08C3F21F4909147021916BCF39FE047
:10260000980F983080F421E030E0A90102C0440F17
:10261000551F9A95E2F7CA0180959091430289234C
:102620008093430213C08D3F21F4809141028E7F3D
:102630000BC08E3F21F4809141028D7F05C08F3FFA
:1026400029F4809141028B7F809341028091440262
:10265000811106C080914502811102C01092400292
:1026600080914602811106C080914702811102C00B
:1026700010923F0208950E94FC17209144022111FC
:1026800004C020914502222321F090933E028093C2
:102690003D0220914602211104C0209147022223CD
:1026A00021F090933C0280933B0282E492E00C94F0
:1026B000D916EF92FF920F931F93CF93DF9300D021
:1026C00000D000D0CDB7DEB786E0E2E4F2E0DE0174
:1026D000119601900D928A95E1F7E0904402F090F6
:1026E0004502009146021091470210924402109256
:1026F00045021092460210924702E11003C0FF20EB
:1027000009F45DC080913D0290913E020E94141830
:10271000AC0190914002992339F020910A0130E0F8
:102720002417350758F04BC020910B018AE0289FF1
:10273000900111242417350718F041C09F3F19F06C
:102740009F5F90934002EE2061F00E94F1111E14F1
:1027500014F09FEF01C091E0989F902D1124909369
:102760004402FF2061F00E94F1111F1414F09FEF4A
:1027700001C091E0989F902D1124909345023091D3
:1027800044023323E1F0209145022223C1F045EBBE
:102790003403C0011124992319F09093440203C01B
:1027A00081E08093440235EB2303C0011124992377
:1027B00019F09093450203C081E080934502011116
:1027C00003C0112309F45DC080913B0290913C024B
:1027D0000E941418AC0190913F02992339F0209186
:1027E000060130E02417350758F04BC0209107014F
:1027F0008AE0289F900111242417350718F041C062
:102800009F3F19F09F5F90933F02002361F00E9469
:102810003012101614F09FEF01C091E0989F902D98
:10282000112490934602112361F00E943012111678
:1028300014F09FEF01C091E0989F902D1124909388
:102840004702309146023323E1F0209147022223D0
:10285000C1F045EB3403C0011124992319F0909382
:10286000460203C081E08093460235EB2303C0019A
:102870001124992319F09093470203C081E08093BB
:1028800047028091440281110BC080914502811161
:1028900007C080914602811103C0809147028111D7
:1028A0000E943B13EB82FC820D831E8386E0FE01B7
:1028B0003196A2E4B2E001900D928A95E1F7269656
:1028C0000FB6F894DEBF0FBECDBFDF91CF911F9141
:1028D0000F91FF90EF900895E2E4F2E086E0DF01CF
:1028E0001D928A95E9F71092400210923F021092D1
:1028F00041020895CF93DF93EC01FB01828188238D
:1029000009F43CC1C430FDE5DF0760F4CB3F9CE532
:10291000D90788F49E0122503C452431310508F046
:102920002EC109C0C236EDE5DE0729F0C63AFDE545
:10293000DF0709F024C10E94B80C909362028093D3
:102940006102C1318CE5D80709F4C6C008F042C065
:10295000C930ECE5DE0709F49BC000F5C5308CE515
:10296000D80709F485C078F4C330ECE5DE0709F434
:1029700078C008F07AC0C230DC4509F0F5C080911B
:1029800061028160EFC0C7309CE5D90709F478C0C7
:1029900008F07AC0809161028061E4C0CD30FCE52E
:1029A000DF0709F487C058F4CB309CE5D90709F458
:1029B00079C008F07BC08091610288606FC0CF3021
:1029C000FCE5DF0709F480C008F082C08091610255
:1029D000877FC8C0CE3F9CE5D90709F471C000F5D8
:1029E000C531FCE5DF0709F485C068F4C3319CE517
:1029F000D90709F475C008F095C00E946906809156
:102A000061028F77AFC0CC3FFCE5DF07A9F108F08A
:102A100054C0CB3FDC4509F0A7C08091620240C0A2
:102A2000C230EDE5DE0709F489C058F4C1158DE523
:102A3000D80709F45AC008F069C080916202826028
:102A40002FC0C236EDE5DE0709F47CC0C63AFDE5CD
:102A5000DF0709F481C0C330DD4509F085C080E09F
:102A60006EC08091610282607DC08091610216C05B
:102A700080916102886076C08091620282604FC05E
:102A80008091610280626EC08091610280646AC040
:102A90000E94690680916102806864C0846062C09F
:102AA00081603DC0809161028E7F5CC08091610237
:102AB0008D7F58C08091610216C08091620218C05B
:102AC000809162028D7F2BC0809161028F7E4AC00F
:102AD000809161028F7D46C0809161028F7B42C0F0
:102AE00080916102877F8B7F3DC0809162028D7FE4
:102AF0008E7F15C08091610282FB222720F991E030
:102B0000922790FB82F990FB83F92CC0809162029E
:102B1000982F909591708E7F892B90FB81F98093EF
:102B2000620222C00E9469068091610287FB22270F
:102B300020F991E0922790FB87F914C081E00E9470
:102B40004F0D12C08091610284FB222720F991E091
:102B5000922790FB84F906C080916102982F90958E
:102B600090FB80F9809361028091610290916202F2
:102B70000E94C90C0E94690680E001C081E0DF91DB
:102B8000CF910895CF93DF9386319C4541F5EB01BA
:102B90000E94BC0B982F8A81209102013091030181
:102BA000882379F09A7A81E009F480E080934802E2
:102BB000911102C069E201C065E3C9010E94551785
:102BC0000AC080914802811102C069E201C065E338
:102BD000C9010E9457170E94FE0B80E001C081E0EE
:102BE000DF91CF9108950F931F93CF93DF93C42F5D
:102BF000D22FFC0182818823C9F040934B020E94AE
:102C0000FC1790934A028093490280E28C0F88302F
:102C100008F057C0C77081E001C0880FCA95EAF775
:102C2000DF91CF911F910F910C94C60380914B02BD
:102C3000481330C08091490290914A020E941418B2
:102C4000883C910538F510E21D0FCD17B9F080E2F0
:102C50008C0F883040F4C77081E001C0880FCA959E
:102C6000EAF70E94CD03183028F581E09D2F977078
:102C700001C0880F9A95EAF70E94C603802F0E9430
:102C8000BD031830F0F4D77081E001C0880FDA95E9
:102C9000EAF70AC080E28C0F883098F4C77081E0B0
:102CA00001C0880FCA95EAF7DF91CF911F910F916C
:102CB0000C94CD03802FDF91CF911F910F910C9435
:102CC000BD03DF91CF911F910F9108950F939C0148
:102CD000CB01243F4CE5340731F188F4293DFCE574
:102CE0003F07D9F02A3D4CE5340779F1283D3C45B2
:102CF000A9F506E221EE41EE68ED7CE52BC0263F0A
:102D0000FCE53F07E1F0A8F0273F3C4539F507E235
:102D100025EE46EE67EF7CE51DC007E225EE45EEA9
:102D200069ED7CE517C006E221EE40EE64EF7CE53C
:102D300011C007E225EE44EE65EF7CE50BC006E22C
:102D400021EE42EE66EF7CE505C008E221E045EEAB
:102D50006AED7CE50E94F31580E008C0FC018281E9
:102D6000882319F010924B0201C081E00F91089561
:102D700090938F0180938E010895909351028093D8
:102D800050020895E0915002F0915102309721F0E5
:102D90000190F081E02D099480E00895E0915002C7
:102DA000F0915102309721F00280F381E02D0994D7
:102DB0000895E0915002F0915102309739F022E0ED
:102DC000DC012C930480F581E02D09940895209175
:102DD0004E0230914F022817390771F090934F023D
:102DE00080934E02E0915002F0915102309721F011
:102DF0000680F781E02D0994089520914C023091CE
:102E00004D022817390771F090934D0280934C02C0
:102E1000E0915002F0915102309721F00084F18549
:102E2000E02D09940895FC01329697E080E09150DE
:102E300029F021912223D9F38F5FF9CF08956623DA
:102E400049F0FC01329608962191621729F0E817A3
:102E5000F907D1F780E0089581E008959C01FC0115
:102E600032969FEF80E04191461789F09F3F19F419
:102E7000411101C0982F8F5F8630A9F79F3F39F02D
:102E8000F901E90FF11D97FDFA9562830895089500
:102E90009C012A5F3F4FFC014281461301C0128210
:102EA000019682179307B9F708950C942E170C9486
:102EB0004817029626E0FC0111922A95E9F7089539
:102EC00008950C94601783E0809352020C9461176C
:102ED000811102C081E001C082E0809352020C9413
:102EE00061170C94681781E0809352020C9461176B
:102EF0000C94731708950C947A170C947B170C9408
:102F00007A170C947A170C947A17CF930E94811732
:102F10000E9452110E947F17C0E08C2F0E947C10EB
:102F2000892B29F4CF5FC930C1F780E001C081E06F
:102F3000CF91089508951F920F920FB60F9211240A
:102F40008F939F93AF93BF9380915302811113C0CE
:102F50008091870290918802A0918902B0918A02A3
:102F60004196A11DB11D8093870290938802A09382
:102F70008902B0938A02BF91AF919F918F910F9078
:102F80000FBE0F901F90189580918F02843031F101
:102F90000E94A1021092530220E488E190E00FB653
:102FA000F894A895809360000FBE2093600083B7CB
:102FB000817F846083BF83B7816083BF7894889565
:102FC00083B78E7F83BF0FB6F894A8958091600079
:102FD000886180936000109260000FBE08950E9487
:102FE00069060C94A50282E084BD93E095BD9AEF3A
:102FF00097BD80936E0008952FB7F8948091870253
:1030000090918802A0918902B0918A022FBF089501
:103010002FB7F8946091870270918802809189029D
:1030200090918A022FBF08959C014FB7F894809128
:10303000870290918802A0918902B0918A024FBFC5
:10304000821B930B089578941F920F920FB60F92E4
:1030500011248F939F93AF93BF9380918702909198
:103060008802A0918902B0918A020196A11DB11D2A
:103070008093870290938802A0938902B0938A027A
:10308000BF91AF919F918F910F900FBE0F901F90A6
:10309000189581E08093E00080E28093D800109240
:1030A000C9008FE19EE40197F1F700C0000087E0BE
:1030B00090EBDC018093980290939902A0939A027E
:1030C000B0939B029CE088E10FB6F894A89580939A
:1030D00060000FBE90936000FFCF80915F02089563
:1030E000089522E02093E9002FEF3091E80021506D
:1030F00035FD06C035ED3A95F1F700002111F5CF09
:103100002091E80025FF0BC040E050E066E070E051
:103110000E949B1A8091E8008E778093E8000895C2
:10312000CF93DF9321E02093E9002FEF3091E80067
:10313000215035FD06C035ED3A95F1F7000021111B
:10314000F5CF2091E80025FF14C0EC0140E050E0ED
:1031500068E070E00E949B1A8091E8008E7780936F
:10316000E80088E0FE01A7E5B2E001900D928A95A3
:10317000E1F7DF91CF910895809354027093560246
:103180006093550280918F02843001F582E0809334
:10319000E9008FEF9091E800815095FD06C095ED14
:1031A0009A95F1F700008111F5CF8091E80085FF35
:1031B0000DC040E050E063E070E084E592E00E94E2
:1031C0009B1A8091E8008E778093E8000895BC01F7
:1031D00084E00C94BC18BC0183E00C94BC18809172
:1031E0008E02811109C00E942C1C0E94891C8091B2
:1031F000E20084608093E200089510928E020895A8
:103200000C94781760918B0281E0611101C080E01D
:103210000C94631790918F0281E0943009F080E064
:1032200060918B020C94681742E061EC81E00E948F
:10323000A51B42E261EC82E00E94A51B90918F02E7
:1032400081E0943009F080E060918B020C9471175A
:1032500080919102833009F461C030F4813071F0C3
:10326000823009F49AC008958A3009F486C08B3000
:1032700009F46CC0893009F0A8C020C08091900288
:10328000813A09F0A2C08091E800877F8093E8002E
:103290008091940290919502892B21F468E087E552
:1032A00092E003C060E080E090E070E00E94E61AE7
:1032B0008091E8008B778093E800089580919002D8
:1032C000813209F082C08091940290919502029718
:1032D00008F07BC08091E800877F8093E8008091B0
:1032E000E80082FD05C080918F028111F8CF6DC08A
:1032F0002091F3008091F20090E0922B029731F43C
:103300008091F100813011F0863021F48091F1003C
:1033100080935F028091E8008B7753C08091900288
:10332000813A09F052C08091940290919502892BC4
:1033300009F04BC08091E800877F8093E80080917E
:10334000E80080FFFCCF8091180136C08091900288
:103350008132D9F58091940290919502892BA9F53B
:103360008091E800877F8093E8000E94DA1B8091BB
:103370009202809318010C94690680919002813228
:1033800021F58091E800877F8093E8000E94DA1B96
:103390008091930280936002089580919002813A17
:1033A000A1F48091E800877F8093E8008091E80095
:1033B00080FFFCCF809160028093F1008091E80053
:1033C0008E778093E8000C94DA1B089584B7877F8A
:1033D00084BF0FB6F894A8958091600088618093AF
:1033E0006000109260000FBE90E080E80FB6F89485
:1033F00080936100909361000FBE0C9473170E943C
:103400002C1C0E94891CE2EEF0E0808184608083A5
:1034100078940C941E1F8CE091E00C94BD16809162
:103420008F028530A9F480918F02853079F40E9453
:10343000C41780918D028823B1F30E9485178823D9
:1034400091F30E94851A0E946906EDCF0C94EF1744
:10345000089508950C942C1A292F33272330310511
:10346000C9F060F42130310581F02230310509F0D6
:1034700044C08BE390E026E532E043C021323105C1
:10348000E1F02232310549F138C082E190E021E9D2
:1034900032E037C099278130910549F028F0029732
:1034A00061F5ECE1F2E005C0E2E5F2E002C0E0E443
:1034B000F2E0849190E09F0124C06115710541F014
:1034C00061307105D1F489E090E021E832E019C063
:1034D00089E090E028E632E014C06115710541F002
:1034E0006130710551F48BE790E023EA32E009C0C6
:1034F00080E490E02EE133E004C080E090E020E042
:1035000030E0FA0131832083089580E189BD82E1B2
:1035100089BD09B400FEFDCF8091D8008F7D8093D6
:10352000D8008091E00082608093E0008091E0000C
:1035300081FDFCCF0895CF92DF92EF92FF920F931F
:103540001F93CF93DF93EC018B017A010E94F91B4B
:10355000811133C0E114F10439F0F70180819181C8
:10356000081B190BC80FD91FC12CD12C011511052F
:1035700019F18091E80085FD16C08091E8008E77F2
:103580008093E800E114F10449F0F7018081918112
:10359000C80ED91ED182C08285E00FC00E94F91BDF
:1035A000882321F30AC089918093F1000150110909
:1035B000FFEFCF1ADF0ADACF80E0DF91CF911F91C2
:1035C0000F91FF90EF90DF90CF9008952091960299
:1035D000309197022617370748F06115710539F4C5
:1035E0002091E8002E772093E80001C0B901FC018A
:1035F00020E06115710579F180918F028823F1F146
:103600008530F1F18091E80083FD3CC08091E800B5
:1036100082FD2EC08091E80080FFEBCF2091F30067
:103620008091F20090E0922B6115710551F0883085
:10363000910538F421912093F100615071090196B0
:10364000F3CF21E0089709F020E08091E8008E7721
:103650008093E800CECF2111CFCF0AC080918F0296
:10366000882361F0853061F08091E80083FD0AC015
:103670008091E80082FFF2CF80E0089582E0089513
:1036800083E0089581E00895209196023091970299
:103690002617370748F06115710539F42091E800C5
:1036A0002E772093E80001C0B901FC0120E06115EC
:1036B000710591F180918F02882309F440C0853013
:1036C00009F43FC08091E80083FD3DC08091E8008F
:1036D00082FD2FC08091E80080FFE9CF2091F300A8
:1036E0008091F20090E0922B6115710559F08830BD
:1036F000910540F424912093F100319661507109B5
:103700000196F2CF21E0089709F020E08091E800CF
:103710008E778093E800CBCF2111CCCF0AC0809167
:103720008F02882361F0853061F08091E80083FD8D
:103730000AC08091E80082FFF2CF80E0089582E025
:10374000089583E0089581E00895982F973068F5F3
:103750009093E900981739F07091EC002091ED00FA
:103760005091F00003C0242F762F50E021FD02C0BD
:103770009F5FECCF3091EB003E7F3093EB003091B8
:10378000ED003D7F3093ED003091EB0031603093E0
:10379000EB007093EC002093ED005093F00020912B
:1037A000EE0027FDE5CF80E008958F708093E9005B
:1037B00081E008958091900287FF11C08091E80018
:1037C00082FD05C080918F028111F8CF11C08091D8
:1037D000E8008B770BC080918F02882349F080919D
:1037E000E80080FFF8CF8091E8008E778093E800B2
:1037F00008952091E4003091E50095E64091EC00B9
:10380000842F817040FF23C08091E80080FD1DC09F
:1038100080918F02882399F0853099F08091EB0098
:1038200085FD11C04091E4005091E5002417350753
:1038300029F3915011F09A01E1CF84E0089582E0DC
:10384000089583E0089581E0089580E0089540910F
:10385000E80042FFDDCF08950E949A1C0E94A21C3E
:10386000E0EEF0E0808181608083E8EDF0E080812F
:103870008F77808319BCA7EDB0E08C918E7F8C93FD
:1038800080818F7E808310928E0208950F931F9304
:10389000CF93DF930E949A1C0E94A21CC8EDD0E037
:1038A00088818F77888388818068888388818F7DED
:1038B000888319BC10928F0210928B0210928D0295
:1038C00010928C0200EE10E0F80180818B7F8083E3
:1038D00088818160888342E060E080E00E94A51BCF
:1038E000E1EEF0E080818E7F8083E2EEF0E0808187
:1038F00081608083808188608083F80180818E7FF1
:103900008083888180618883DF91CF911F910F919F
:103910000895E8EDF0E080818F7E8083E7EDF0E0B0
:1039200080818160808384E082BF81E080938E0209
:103930000C94461CE8EDF0E080818E7F808310922D
:10394000E20008951092DA001092E10008951F92AB
:103950000F920FB60F9211242F933F934F935F93C3
:103960006F937F938F939F93AF93BF93EF93FF9347
:103970008091E10082FF0BC08091E20082FF07C0CE
:103980008091E1008B7F8093E1000E941D1F809158
:10399000DA0080FF1FC08091D80080FF1BC080919B
:1039A000DA008E7F8093DA008091D90080FF0DC00D
:1039B00080E189BD82E189BD09B400FEFDCF81E0CF
:1039C00080938F020E94EF1805C019BC10928F02DD
:1039D0000E94FD188091E10080FF19C08091E200F3
:1039E00080FF15C08091E2008E7F8093E20080917D
:1039F000E20080618093E2008091D8008062809331
:103A0000D80019BC85E080938F020E940219809132
:103A1000E10084FF30C08091E20084FF2CC080E18F
:103A200089BD82E189BD09B400FEFDCF8091D80037
:103A30008F7D8093D8008091E1008F7E8093E1009C
:103A40008091E2008F7E8093E2008091E2008160AD
:103A50008093E20080918B02882311F084E007C0FC
:103A60008091E30087FD02C081E001C083E0809384
:103A70008F020E940A198091E10083FF29C0809182
:103A8000E20083FF25C08091E100877F8093E10001
:103A900082E080938F0210928B028091E1008E7FF2
:103AA0008093E1008091E2008E7F8093E20080911C
:103AB000E20080618093E20042E060E080E00E94EA
:103AC000A51B8091F00088608093F0000E9400198F
:103AD000FF91EF91BF91AF919F918F917F916F91E6
:103AE0005F914F913F912F910F900FBE0F901F90BC
:103AF00018951F920F920FB60F9211242F933F9398
:103B00004F935F936F937F938F939F93AF93BF93E5
:103B1000CF93DF93EF93FF93C091E900CF70809133
:103B2000EC00D82FD17080FDD0E81092E900809190
:103B3000F000877F8093F00078940E94BD1D109262
:103B4000E9008091F00088608093F000CD2BCF7069
:103B5000C093E900FF91EF91DF91CF91BF91AF91B9
:103B60009F918F917F916F915F914F913F912F9195
:103B70000F900FBE0F901F9018951F93CF93DF9358
:103B8000CDB7DEB7AA970FB6F894DEBF0FBECDBF94
:103B9000E0E9F2E08091F100819322E0E839F20758
:103BA000C9F70E9428198091E80083FF2EC18091F7
:103BB000900290919102492F50E04A30510508F04F
:103BC00024C1FA01EE59FF4F0C944D1F803821F0AB
:103BD000823809F01AC108C080918C0290918D0240
:103BE000992389F082600FC0809194028F70873092
:103BF00008F00BC18093E9008091EB0085FB8827DA
:103C000080F91092E9009091E800977F9093E80086
:103C10008093F1001092F100D1C0282F2D7F09F080
:103C2000F4C0882319F0823061F0EFC080919202D5
:103C3000813009F0EAC0933009F080E080938D0272
:103C40002EC08091920281112AC0809194028F70BF
:103C50002FEF280F263008F0D8C08093E90020917C
:103C6000EB0020FF1CC0933021F48091EB008062B8
:103C700014C09091EB0090619093EB0021E030E054
:103C8000A90102C0440F551F8A95E2F74093EA004C
:103C90001092EA008091EB0088608093EB00109214
:103CA000E9008091E800877F8093E8000E94DA1B9A
:103CB000ACC08111AAC0109192021F778091E300DD
:103CC0008078812B8093E3008091E800877F809348
:103CD000E8000E94DA1B8091E80080FFFCCF809111
:103CE000E30080688093E300111102C082E001C00C
:103CF00083E080938F0289C08058823008F085C0AD
:103D000080919202909193028C3D53E0950779F552
:103D100083E08A838AE289834FB7F894DE011396A1
:103D200020E03EE051E2E32FF0E050935700E491B1
:103D300020FF03C0E295EF703F5FEF708E2F90E0A1
:103D4000EA3010F0C79601C0C0968D939D932F5F07
:103D5000243149F74FBF8091E800877F8093E800C6
:103D60006AE270E0CE0101960E94E61A16C06091E8
:103D7000940270919502AE014F5F5F4F0E942A1A24
:103D8000BC01892B09F441C09091E800977F909382
:103D9000E80089819A810E94441B8091E8008B771A
:103DA0008093E80032C0803881F58091E800877FF9
:103DB0008093E80080918B028093F1008091E8006D
:103DC0008E7772CF811121C08091920290919302DF
:103DD00099270297D4F48091E800877F8093E800C8
:103DE0008091920280938B020E94DA1B80918B0259
:103DF000811106C08091E30087FD02C081E001C00F
:103E000084E080938F020E9414198091E80083FF60
:103E10000AC08091E800877F8093E8008091EB00E2
:103E200080628093EB00AA960FB6F894DEBF0FBEB7
:103E3000CDBFDF91CF911F9108950895CF938091C9
:103E40008F028823A1F0C091E900CF709091EC001F
:103E5000892F817090FD80E8C82B1092E900809135
:103E6000E80083FD0E94BD1DCF70C093E900CF9193
:103E7000089597FB072E16F4009407D077FD09D01C
:103E80000E94531F07FC05D03EF4909581959F4FEB
:103E90000895709561957F4F0895EE0FFF1F05906F
:103EA000F491E02D0994AA1BBB1B51E107C0AA1F86
:103EB000BB1FA617B70710F0A61BB70B881F991FCB
:103EC0005A95A9F780959095BC01CD010895FB0105
:103ED000DC0104C08D910190801921F441505040C3
:103EE000C8F7881B990B0895F999FECF92BD81BD43
:103EF000F89A992780B50895A8E1B0E042E050E033
:103F00000C94A81F262FF999FECF92BD81BDF89A77
:103F1000019700B4021639F01FBA20BD0FB6F8940D
:103F2000FA9AF99A0FBE08950396272F0E94831FCD
:103F30000E94821F252F0E94831F242F0C94831F11
:103F40000196272F0E94831F0C94821FDC01CB0156
:103F5000FC01F999FECF06C0F2BDE1BDF89A319699
:103F600000B40D9241505040B8F70895F894FFCF37
:103F7000C8001302280850011E0A14016D18901879
:103F80007118EB18E718701801E200E900EA00B5B3
:103F900000B600B700CD008301CC008A01920194E5
:103FA000012102230224022502260227022A02B34B
:103FB00000B4006F007000818283E200E900EA0033
:103FC000B500B600B700CD008301CC008A01920194
:103FD00094012102230224022502260227022A023A
:103FE000B300B4006F00700081828336F7F6F5F4F9
:0E3FF0009091973432F0669493F192359500DB
:00000001FF
